 adc

 Timestamp is 4fb05c69 (Mon May 14 13:14:17 2012)

 Preferred load address is 10000000

 Start         Length     Name                   Class
 0001:00000000 00000004H .CRT$XCA                CODE
 0001:00000004 00000004H .CRT$XCZ                CODE
 0001:00000008 00000004H .CRT$XIA                CODE
 0001:0000000c 00000004H .CRT$XIZ                CODE
 0001:00000010 00000004H .CRT$XPA                CODE
 0001:00000014 00000004H .CRT$XPZ                CODE
 0001:00000018 00000004H .CRT$XTA                CODE
 0001:0000001c 00000004H .CRT$XTZ                CODE
 0001:00000020 00000288H .rdata                  CODE
 0001:000002a8 00000020H .rdata$debug            CODE
 0001:000002c8 00001d9cH .text                   CODE
 0001:00002064 0000005cH .xdata                  CODE
 0001:000020c0 0000003cH .idata$2                CODE
 0001:000020fc 00000014H .idata$3                CODE
 0001:00002110 00000078H .idata$4                CODE
 0001:00002188 0000004cH .idata$6                CODE
 0001:000021e0 00000106H .edata                  CODE
 0002:00000000 00000078H .idata$5                DATA
 0002:00000078 00000008H .data                   DATA
 0002:00000080 00000014H .bss                    DATA
 0003:00000000 00000130H .pdata                  DATA

  Address         Publics by Value              Rva+Base       Lib:Object

 0000:00000000       ___safe_se_handler_count   00000000     <absolute>
 0000:00000000       ___safe_se_handler_table   00000000     <absolute>
 0001:00000000       __xc_a                     10001000     corelib0:crt0init.obj
 0001:00000004       __xc_z                     10001004     corelib0:crt0init.obj
 0001:00000008       __xi_a                     10001008     corelib0:crt0init.obj
 0001:0000000c       __xi_z                     1000100c     corelib0:crt0init.obj
 0001:00000010       __xp_a                     10001010     corelib0:crt0init.obj
 0001:00000014       __xp_z                     10001014     corelib0:crt0init.obj
 0001:00000018       __xt_a                     10001018     corelib0:crt0init.obj
 0001:0000001c       __xt_z                     1000101c     corelib0:crt0init.obj
 0001:000000d0       ??_C@_1DA@PPMNHOKM@?$AAA?$AAD?$AAC?$AA?5?$AA?3?$AA?5?$AAI?$AAn?$AAv?$AAa?$AAl?$AAi?$AAd?$AA?5?$AAI?$AAP?$AAG?$AA?5?$AAC?$AAl?$AAk?$AA?$AN?$AA?6?$AA?$AA@ 100010d0     adc_common_topaz_v1:adc.obj
 0001:00000100       ??_C@_1CI@OHCJFJPM@?$AAE?$AAR?$AAR?$AAO?$AAR?$AA?3?$AA?5?$AA?$CF?$AAs?$AA?5?$AAl?$AAi?$AAn?$AAe?$AA?5?$AA?$CF?$AAd?$AA?3?$AA?5?$AA?$AA@ 10001100     adc_common_topaz_v1:adc.obj
 0001:00000128       ??_C@_1KK@DJNGEBAF@?$AAC?$AA?3?$AA?2?$AAW?$AAI?$AAN?$AAC?$AAE?$AAR?$AAO?$AAO?$AAT?$AAS?$AA?2?$AAT?$AAo?$AAp?$AAa?$AAz?$AA?2?$AAW?$AAI?$AAN?$AAC?$AAE?$AA6?$AA0?$AA0?$AA?2?$AAP?$AAL?$AAA@ 10001128     adc_common_topaz_v1:adc.obj
 0001:000001d8       ??_C@_1EG@BODOANKG@?$AAE?$AAx?$AAc?$AAe?$AAp?$AAt?$AAi?$AAo?$AAn?$AA?5?$AAi?$AAn?$AA?5?$AAA?$AAD?$AAC?$AA?5?$AAI?$AAO?$AAC?$AAT?$AAL?$AA_?$AAP?$AAO?$AAW?$AAE?$AAR?$AA_?$AAS?$AAE?$AAT@ 100011d8     adc_common_topaz_v1:adc.obj
 0001:00000220       ??_C@_1FK@CFOKMKHC@?$AAE?$AAx?$AAc?$AAe?$AAp?$AAt?$AAi?$AAo?$AAn?$AA?5?$AAi?$AAn?$AA?5?$AAD?$AAV?$AAF?$AAC?$AA?5?$AAI?$AAO?$AAC?$AAT?$AAL?$AA_?$AAP?$AAO?$AAW?$AAE?$AAR?$AA_?$AAC?$AAA@ 10001220     adc_common_topaz_v1:adc.obj
 0001:0000027c       ??_C@_1CM@GMJLMKBF@?$AAn?$AAo?$AAt?$AA?5?$AAi?$AAm?$AAp?$AAl?$AAe?$AAm?$AAe?$AAn?$AAt?$AAe?$AAd?$AA?5?$AAy?$AAe?$AAt?$AA?$AN?$AA?6?$AA?$AA@ 1000127c     adc_common_topaz_v1:adc.obj
 0001:000002c8       BSPADCCIomuxConfig         100012c8 f   adc.obj
 0001:000002e0       BSPADCEnableClock          100012e0 f   adc.obj
 0001:00000348       BSPADCGetIPGClock          10001348 f   adc.obj
 0001:00000374       BSPADCGetHSYNCPolarity     10001374 f   adc.obj
 0001:0000038c       BSPADCGetHSYNCEnable       1000138c f   adc.obj
 0001:000003a4       ADC_Deinit                 100013a4 f   adc_common_topaz_v1:adc.obj
 0001:00000414       ADC_Init                   10001414 f   adc_common_topaz_v1:adc.obj
 0001:0000064c       ADC_Open                   1000164c f   adc_common_topaz_v1:adc.obj
 0001:000006ac       ADC_Close                  100016ac f   adc_common_topaz_v1:adc.obj
 0001:000006f8       ADC_IOControl              100016f8 f   adc_common_topaz_v1:adc.obj
 0001:00001570       ADC_Read                   10002570 f   adc_common_topaz_v1:adc.obj
 0001:00001598       ADC_Write                  10002598 f   adc_common_topaz_v1:adc.obj
 0001:000015c0       ADC_Seek                   100025c0 f   adc_common_topaz_v1:adc.obj
 0001:000015e8       ADC_PowerUp                100025e8 f   adc_common_topaz_v1:adc.obj
 0001:000015fc       ADC_PowerDown              100025fc f   adc_common_topaz_v1:adc.obj
 0001:00001610       LocalFree                  10002610 f   coredll:COREDLL.dll
 0001:00001620       DeleteCriticalSection      10002620 f   coredll:COREDLL.dll
 0001:00001630       NKDbgPrintfW               10002630 f   coredll:COREDLL.dll
 0001:00001640       Sleep                      10002640 f   coredll:COREDLL.dll
 0001:00001650       InitializeCriticalSection  10002650 f   coredll:COREDLL.dll
 0001:00001660       LocalAlloc                 10002660 f   coredll:COREDLL.dll
 0001:00001670       GetTickCount               10002670 f   coredll:COREDLL.dll
 0001:00001680       LeaveCriticalSection       10002680 f   coredll:COREDLL.dll
 0001:00001690       EnterCriticalSection       10002690 f   coredll:COREDLL.dll
 0001:000016a0       SetLastError               100026a0 f   coredll:COREDLL.dll
 0001:000016b0       MmUnmapIoSpace             100026b0 f   ceddk:CEDDK.dll
 0001:000016c0       MmMapIoSpace               100026c0 f   ceddk:CEDDK.dll
 0001:000016d0       DDKClockSetGatingMode      100026d0 f   cspddk:CSPDDK.dll
 0001:000016e0       DDKClockGetFreq            100026e0 f   cspddk:CSPDDK.dll
 0001:000016f0       DllMain                    100026f0 f   corelib0:dllmain.obj
 0001:0000172c       _DllMainCRTStartup         1000272c f   corelib0:pegdmain.obj
 0001:000018d4       __security_init_cookie     100028d4 f   corelib0:seccinit.obj
 0001:0000199c       exit                       1000299c f   corelib0:cexit.obj
 0001:00001b1c       _exit                      10002b1c f   corelib0:cexit.obj
 0001:00001b40       _cexit                     10002b40 f   corelib0:cexit.obj
 0001:00001b5c       _c_exit                    10002b5c f   corelib0:cexit.obj
 0001:00001b78       GetCurrentProcess          10002b78 f i corelib0:cexit.obj
 0001:00001b90       _initterm                  10002b90 f   corelib0:crt0dat.obj
 0001:00001be4       _cinit                     10002be4 f   corelib0:crt0dat.obj
 0001:00001c20       _onexit                    10002c20 f   corelib0:onexit.obj
 0001:00001f24       atexit                     10002f24 f   corelib0:onexit.obj
 0001:00001f78       __rt_udiv                  10002f78 f   corelib1:COREDLL.dll
 0001:00001f88       memset                     10002f88 f   corelib1:COREDLL.dll
 0001:00001f98       __C_specific_handler       10002f98 f   corelib1:COREDLL.dll
 0001:00001fa8       _XcptFilter                10002fa8 f   corelib1:COREDLL.dll
 0001:00001fb8       __security_gen_cookie2     10002fb8 f   corelib1:COREDLL.dll
 0001:00001fc8       free                       10002fc8 f   corelib1:COREDLL.dll
 0001:00001fd8       malloc                     10002fd8 f   corelib1:COREDLL.dll
 0001:00001fe8       realloc                    10002fe8 f   corelib1:COREDLL.dll
 0001:00001ff8       _msize                     10002ff8 f   corelib1:COREDLL.dll
 0001:00002008       CspADCTouchGetBaseRegAddr  10003008 f   adc_mx25_topaz_v1:adc.obj
 0001:00002024       DisableThreadLibraryCalls  10003024 f   coredll:COREDLL.dll
 0001:00002034       InterlockedExchange        10003034 f   coredll:COREDLL.dll
 0001:00002044       TerminateProcess           10003044 f   coredll:COREDLL.dll
 0001:00002054       InterlockedCompareExchange 10003054 f   coredll:COREDLL.dll
 0001:000020c0       __IMPORT_DESCRIPTOR_COREDLL 100030c0     coredll:COREDLL.dll
 0001:000020d4       __IMPORT_DESCRIPTOR_CEDDK  100030d4     ceddk:CEDDK.dll
 0001:000020e8       __IMPORT_DESCRIPTOR_CSPDDK 100030e8     cspddk:CSPDDK.dll
 0001:000020fc       __NULL_IMPORT_DESCRIPTOR   100030fc     coredll:COREDLL.dll
 0002:00000000       __imp_MmUnmapIoSpace       10004000     ceddk:CEDDK.dll
 0002:00000004       __imp_MmMapIoSpace         10004004     ceddk:CEDDK.dll
 0002:00000008       \177CEDDK_NULL_THUNK_DATA  10004008     ceddk:CEDDK.dll
 0002:0000000c       __imp_Sleep                1000400c     coredll:COREDLL.dll
 0002:00000010       __imp_InitializeCriticalSection 10004010     coredll:COREDLL.dll
 0002:00000014       __imp_LocalAlloc           10004014     coredll:COREDLL.dll
 0002:00000018       __imp_NKDbgPrintfW         10004018     coredll:COREDLL.dll
 0002:0000001c       __imp_LeaveCriticalSection 1000401c     coredll:COREDLL.dll
 0002:00000020       __imp_EnterCriticalSection 10004020     coredll:COREDLL.dll
 0002:00000024       __imp_SetLastError         10004024     coredll:COREDLL.dll
 0002:00000028       __imp_DeleteCriticalSection 10004028     coredll:COREDLL.dll
 0002:0000002c       __imp_GetTickCount         1000402c     coredll:COREDLL.dll
 0002:00000030       __imp_LocalFree            10004030     coredll:COREDLL.dll
 0002:00000034       __imp_TerminateProcess     10004034     coredll:COREDLL.dll
 0002:00000038       __imp_InterlockedCompareExchange 10004038     coredll:COREDLL.dll
 0002:0000003c       __imp_InterlockedExchange  1000403c     coredll:COREDLL.dll
 0002:00000040       __imp___rt_udiv            10004040     corelib1:COREDLL.dll
 0002:00000044       __imp_memset               10004044     corelib1:COREDLL.dll
 0002:00000048       __imp___C_specific_handler 10004048     corelib1:COREDLL.dll
 0002:0000004c       __imp__XcptFilter          1000404c     corelib1:COREDLL.dll
 0002:00000050       __imp___security_gen_cookie2 10004050     corelib1:COREDLL.dll
 0002:00000054       __imp_free                 10004054     corelib1:COREDLL.dll
 0002:00000058       __imp_malloc               10004058     corelib1:COREDLL.dll
 0002:0000005c       __imp_realloc              1000405c     corelib1:COREDLL.dll
 0002:00000060       __imp__msize               10004060     corelib1:COREDLL.dll
 0002:00000064       __imp_DisableThreadLibraryCalls 10004064     coredll:COREDLL.dll
 0002:00000068       \177COREDLL_NULL_THUNK_DATA 10004068     coredll:COREDLL.dll
 0002:0000006c       __imp_DDKClockSetGatingMode 1000406c     cspddk:CSPDDK.dll
 0002:00000070       __imp_DDKClockGetFreq      10004070     cspddk:CSPDDK.dll
 0002:00000074       \177CSPDDK_NULL_THUNK_DATA 10004074     cspddk:CSPDDK.dll
 0002:00000078       __security_cookie          10004078     corelib0:seccinit.obj
 0002:0000007c       __security_cookie_complement 1000407c     corelib0:seccinit.obj
 0002:00000080       _exitflag                  10004080     corelib0:cexit.obj
 0002:00000084       __onexitend                10004084     <common>
 0002:00000088       __onexitbegin              10004088     <common>
 0002:0000008c       g_pcsExit                  1000408c     <common>
 0002:00000090       _pRawDllMain               10004090     <common>

 entry point at        0001:0000172c

 Static symbols

 0001:00001780       _DllMainCRTStartupHelper   10002780 f   corelib0:pegdmain.obj
 0001:000019c0       doexit                     100029c0 f   corelib0:cexit.obj
 0001:00001c7c       lockexit                   10002c7c f   corelib0:onexit.obj
 0001:00001d18       unlockexit                 10002d18 f   corelib0:onexit.obj
 0001:00001d44       _onexit_nolock             10002d44 f   corelib0:onexit.obj
